:100000000C9496010C94BE010C94BE010C94BE019C
:100010000C94BE010C94BE010C94BE010C94BE0164
:100020000C94BE010C9424020C94B8210C946A2008
:100030000C94BE010C94BE010C94BE010C94BE0144
:100040000C943E090C94BE010C94BE010C94BE01AC
:100050000C94BE010C94BE010C94BE010C949D182E
:100060000C94BE010C945F1D0C94A21D0C94BE0157
:100070000C94BE010C94BE010C94BE010C94BE0104
:100080000C94BE010C94BE010C94BE010C94BE01F4
:100090000C94BE010C94BE010C94BE010C94BE01E4
:1000A0000C94BE010C94BE010C94BE015211581167
:1000B0005E11651173119511B311A619A9199C1937
:1000C000A019CA19CA19CA19AD19B119B519BB199C
:1000D000BF19CA19C519434C49206E6F7420617647
:1000E00061696C61626C652C2075736520636F6E4D
:1000F000666967757261746F72210000000002000A
:10010000080E0000030401000B00000000000000C6
:100110000000000000000000000408020110408000
:1001200040102040804080080204018040201002DE
:10013000011080102040400404040404030405025C
:100140000202020403020202020606060606060472
:100150000402020204000000002300260029002CF3
:10016000002F0000000000250028002B002E003189
:100170000000000000240027002A002D00300008A5
:100180000B0002020201000904000001020200004B
:1001900005240010010524010101042402060524A0
:1001A0000600010705810310004009040100020A4E
:1001B000000000070502024000000705830240001E
:1001C0000000C18081C112010002020000404123F1
:1001D000368000010102000112010002000000400F
:1001E0004123368000010102000118034100720022
:1001F0006400750069006E006F0020004C004C0028
:1002000043002203410072006400750069006E0023
:100210006F0020004C0065006F006E0061007200EE
:1002200064006F00040309040000000000000000E7
:100230002A2B280000000000000000000000000041
:1002400000000000000000002C9EB4A0A1A2A43475
:10025000A6A7A5AE362D3738271E1F20212223241E
:100260002526B333B62EB7B89F8485868788898ABA
:100270008B8C8D8E8F909192939495969798999A56
:100280009B9C9D2F3130A3AD350405060708090A54
:100290000B0C0D0E0F101112131415161718191A36
:1002A0001B1C1DAFB1B0B500090402000103000022
:1002B00000092101010001226500070584034000B7
:1002C0000105010902A1010901A100850105091922
:1002D000012903150025019503750181029501751A
:1002E00005810305010930093109381581257F751C
:1002F0000895038106C0C005010906A10185020514
:100300000719E029E7150025017501950881029577
:1003100001750881039506750815002565050719FF
:100320000029658100C0571B901E542311241FBE55
:10033000CFEFDAE0DEBFCDBF12E0A0E0B1E0E4E550
:10034000F9E402C005900D92AC32B107D9F714E080
:10035000ACE2B2E001C01D92A93EB107E1F713E0A3
:10036000CCE2D3E004C02297FE010E941D24C632D5
:10037000D107C9F70E94CC1E0C94A8240C9400004D
:1003800080910008909101088737974709F0A89558
:100390000895DC01ED91FC910190F081E02D09952B
:1003A00008958091CD03813019F482E08093CD03CC
:1003B0008091CD03833019F484E08093CD030895B8
:1003C00088E08093C10061E08AE00E94CB1960E080
:1003D0008AE00E94041A08950097C9F09C0140E049
:1003E00050E068E478EE81E090E00E94C5232F3F62
:1003F00031054105510529F020F02FEF30E040E0B4
:1004000050E02093D1008091C000806103C08091B2
:10041000C0008F7E8093C0000895219A229A23986D
:1004200060E08BE00E94CB1961E08CE00E94CB1968
:100430000895EBE6F0E0808180688083E8E6F0E0F4
:1004400080818160808308951F920F920FB60F9272
:1004500011242F933F934F935F936F937F938F93C9
:100460009F93AF93BF93EF93FF931F9B0E94D10184
:10047000FF91EF91BF91AF919F918F917F916F917C
:100480005F914F913F912F910F900FBE0F901F9052
:100490001895A1E0B0E0EFE4F2E00C94F3231FB76D
:1004A00091E09093CC03F89489830E94C00198E175
:1004B0009093600089818093600081110E94C00147
:1004C0001FBF2196E3E00C940F2420916C03309120
:1004D0006D03382748E0C901880F991F37FF06C010
:1004E0009C0151E2252750E1352701C09C01415074
:1004F00091F730936D0320936C030895D82FC0E0DB
:10050000CD1780F45F9A64E670E080E090E00E948E
:1005100016195F9864E670E080E090E00E9416197A
:10052000CF5FEECF6CE271E080E090E00E941619A0
:10053000E6CF0F931F93CF93DF93EC01062F15E0C7
:10054000115051F0CE010E949224081741F0602F03
:10055000CE010E949A24F4CF82E00E947E02DF91B5
:10056000CF911F910F910895A0E0B0E0EAEBF2E087
:100570000C94E623482E562EC0E0D0E0612C712C5E
:10058000E12CF12C00E010E041100CC06090CB0396
:1005900086E4689E30011124A9E1EA2EF12C02EBD9
:1005A00013E01EC091E049120FC06090CB03E6E457
:1005B0006E9E30011124FBE16F0E711CF9E2EF2EEB
:1005C000F12C0EE613E00CC082E0481209C078E17D
:1005D000672E77247394EE24E394F12C0BEC13E054
:1005E00043018C0E9D1E10926D0310926C0334011A
:1005F000A62CA818B12CC30101966C01AE14BF043F
:10060000A8F4A00EB11E511006C0C3010E9492248E
:10061000F501808305C0F5016081C3010E94990244
:10062000F50180810E9465023601E2CFC3015110BD
:1006300018C0C3010E949224B82EC6010E949224C1
:100640002B2D30E0322F2227282B80916C039091A4
:100650006D038217930779F4C0E0D0E055245394DA
:1006600093CF360160916D030E94990260916C03F3
:10067000C6010E949902C05EDE4FC13E92E0D907DA
:1006800008F482CF852DCDB7DEB7E0E10C940224CB
:1006900087E380936E0380E092ECA1E0B0E080936A
:1006A0006F0390937003A0937103B093720387E07C
:1006B00080937B0380EC9AECA9E8B6E38093730304
:1006C00090937403A0937503B093760385E08093B1
:1006D0007C038DEE9EEFADEABEED809377039093A1
:1006E0007803A0937903B0937A03EDE7F3E080E019
:1006F00090E0863028F4DC01AA50BE4F2C9101C056
:1007000020E0219301968831910599F782E080934A
:1007100095038AE080939603089561E082E00E9449
:10072000B402089560E082E00E94B4028091CB039D
:10073000843020F01092CB030E948D030895A1E035
:10074000B0E0E5EAF3E00C94F42389830E9492037D
:100750009091CB038981981731F0843020F48093F5
:10076000CB030E948D032196E2E00C94102480ECD0
:1007700097EFAAEBB7E38093B3039093B403A093EE
:10078000B503B093B60380E090E0A0E0B0E58093BD
:10079000B7039093B803A093B903B093BA03EBEBFC
:1007A000F3E080E081938F5F8031E1F70895A0E06E
:1007B000B0E0EDEDF3E00C94EA230E94F31861152C
:1007C000710581059105C9F30E9489241092770370
:1007D000109278031092790310927A03C4E0C12C2E
:1007E000D12C7601CA948090770390907803A090E2
:1007F0007903B0907A03BA2CA92C982C88240E94F3
:100800008424A70196010E94C523680D791D8A1DC5
:100810009B1D609377037093780380937903909383
:100820007A03C15001F70DE713E0E801C12CD12C88
:10083000B2E38B2E912CA12CB12C80E1E82E87E223
:10084000F82E8881882309F446C0D39419F40E94B5
:10085000480341C00E948424A50194010E94C5233D
:1008600021E0260FEDE7F3E08E2F801B8C1520F49E
:1008700081918213F9CFE9CF40917C03249FA0019D
:1008800011244E9DC0014F9D900D5E9D900D112431
:10089000AA2797FDA095BA2F409173035091740336
:1008A0006091750370917603840F951FA61FB71F83
:1008B0004091B3035091B4036091B5037091B603B6
:1008C000481759076A077B0708F4BFCF2993C394D9
:1008D00088E1C812B6CFCDB7DEB7ECE00C940624A1
:1008E00061E080E00E94B40261E081E00E94B40215
:1008F000089560E080E00E94B402882331F060E057
:1009000081E00E94B402811108C00E94B7030E94D6
:1009100048030E94D7030E94700408958F929F920B
:10092000AF92BF92CF92DF92EF92FF92CF93FC01F2
:10093000C0A5EC2FE770F0E0E251FE4FA081B0E0DF
:10094000C7FF03C024E130E002C02FE030E0FC012B
:1009500097A183E1989FF0011124E25CFE4F808013
:100960009180A280B380A20FB31F20E43FE14DE746
:1009700050E00E947723A50194010E94A3238C2FAD
:10098000887149F469017A01E0EDCE0EE7E0DE1EE0
:10099000E11CF11C1BC0C7FF05C060E47AE88CE2D3
:1009A0009EE004C060E07EEE8AEB9BE069017A0184
:1009B000F8EBCF0EFBE0DF1EE11CF11CA50194015A
:1009C0000E94A323C20ED31EE41EF51EC701B6016A
:1009D00069517C4F8F4F9F4F28EE33E040E050E04D
:1009E0000E94A323A8EEB3E00E946C23CF91FF9056
:1009F000EF90DF90CF90BF90AF909F908F90089531
:100A00008F3F910551F048F0811522E0920738F0B0
:100A10008115934030F482E0089580E0089581E0EC
:100A2000089583E00895A0E0B0E0E9E1F5E00C94DA
:100A3000EF23EB018A01B82FB695A0E02881398118
:100A4000F80120832A813B8121832C813D812283EF
:100A50002E813F812383688179814A815B812C814A
:100A60003D81EE81FF819F2F9295990F990F907C88
:100A7000272F2370922B252F2370220F220F922BCA
:100A8000232F23702295207F922BF80194830B5FF4
:100A90001F4F2896AF5FBA1788F680FF24C0888161
:100AA00099810E940005D82E8A819B810E940005B1
:100AB000E82E8C819D810E940005F82E8E819F81F9
:100AC0000E940005F0E4DF9EA001112490E1E99E60
:100AD00090011124242B282BE4E0FE9EB001112468
:100AE000262BF8012083CDB7DEB7E7E00C940B246A
:100AF000803223E0920708F1883E23E0920740F419
:100B00008F519340E4E096958795EA95E1F7089533
:100B1000803D27E0920718F48C5D93400895883952
:100B200028E0920768F4885C974074E09695879572
:100B30007A95E1F78D509C4F089580E090E00895FC
:100B40008FEF93E008958C30910540F4A4E0880F76
:100B5000991FAA95E1F7885D9C4F0895843F23E093
:100B6000920718F484529C4F0895811524E092074F
:100B700040F48657934FF4E0880F991FFA95E1F7F8
:100B8000089580E998E008959C013695279525758C
:100B90003575821B930B9C01237333739695879550
:100BA0009695879583739373820F931F9C0154E0EE
:100BB000369527955A95E1F7280F391F2F703F700A
:100BC00041E051E0249FC001259F900D349F900D7E
:100BD0001124892F08952998882319F000002A9A52
:100BE00002C000002A980000299A00000895299A5E
:100BF000000083B12998000083FB882780F90895BD
:100C0000CF93DF93D82F5E9A29985E98C8E08D2FF6
:100C100080780E94EB05DD0FC150C9F72998DF915C
:100C2000CF9108958F770E9400060895CF93DF93A8
:100C3000D82FC8E08D2F80780E94EB05DD0FC150C2
:100C4000C9F72998DF91CF910895CF93DF93299821
:100C5000C8E080E0D82FDD0F0E94F7058D0FC1504E
:100C6000C9F7DF91CF9108950E9412060E942506D0
:100C70005E9A0895A1E0B0E0E0E4F6E00C94F4237D
:100C8000806869830E9400066981862F0E9416068B
:100C90005E9A2196E2E00C941024CF93C0917703E2
:100CA000C827E82FF0E0E259FC4F678589E70E94EA
:100CB0003A066C2F8DE30E943A066C2F82E40E9464
:100CC0003A06CF91089586E20E9434060895CF93A4
:100CD000DF93EC016C818CE10E943A066D818DE11D
:100CE0000E943A066E818EE10E943A066F8180E290
:100CF0000E943A06688581E20E943A06698582E28E
:100D00000E943A066A8583E20E943A066B8584E275
:100D10000E943A066C8585E20E943A066D858AE259
:100D20000E943A066E858EE60E943A066F858FE62F
:100D30000E943A06688980E70E943A06698981E73D
:100D40000E943A066A8982E70E943A06DF91CF91B3
:100D50000895CF92DF92EF92FF92CF93DF936B01D2
:100D60007C01C11488E3D8068CE9E8068CE1F8061A
:100D700028F5C701B60120E836E948E950E00E94AD
:100D8000A323E901689760E879E687E69FEF0E9470
:100D90007F236C0D7D1D8E1D9F1DF2E0660F771F5A
:100DA000881F991FFA95D1F721E732E040E050E023
:100DB0000E94A323F22EE32E80E421C0C701B601D6
:100DC00020E03DE241E351E00E94A323E90168975E
:100DD00060E073ED8EEC9EEF0E947F236C0D7D1D15
:100DE0008E1D9F1D660F771F881F991F21E732E018
:100DF00040E050E00E94A323F22EE32E80E66C2F09
:100E00006F71680F85E70E943A066E2D86E70E9493
:100E10003A066F2D87E70E943A06DF91CF91FF9047
:100E2000EF90DF90CF900895682F8DE60E943A06EC
:100E300008958F929F92AF92BF92CF92DF92EF92DE
:100E4000FF92CF93DF93D82F83E00E9434068093E4
:100E50006B0384E00E94340680936A0360E086E0BE
:100E60000E943A0661E087E00E943A066FE789E057
:100E70000E943A0665E08AE00E943A0665E18BE04E
:100E80000E943A0662E18CE00E943A066DEF8DE026
:100E90000E943A0660E08EE00E943A06DD2319F0D7
:100EA0008BE291E008C02091950333E1239FC001BC
:100EB0001124825C9E4F0E9467066CE880E30E94CA
:100EC0003A066FE082E30E943A0662E483E30E94FE
:100ED0003A068091960387FF02C064E101C06AE090
:100EE00084E30E943A066AE285E30E943A066DE2D4
:100EF00086E30E943A0664ED87E30E943A0660E0CA
:100F000088E30E943A0660E089E30E943A06D11124
:100F100009C0C0907703D0907803E0907903F090F7
:100F20007A0307C0C5E8CC2EC1ECDC2EED2CCEED4B
:100F3000FC2ECAE38F2C9924AA24BB24682D8C2F65
:100F40000E943A06682D85E08C0F0E943A06FE2C1E
:100F5000ED2CDC2CCC24CF5FCE3361F76FEF83E434
:100F60000E943A066FEF84E40E943A066FEF85E430
:100F70000E943A066FEF86E40E943A06DD2311F0E4
:100F800066E002C060917B038DE60E943A0660E055
:100F900089E70E943A0660917C038AE70E943A063C
:100FA00060E083E70E943A0660E084E70E943A0628
:100FB000D11109C06091730370917403809175031E
:100FC0009091760304C060EC7AEC89E896E30E9485
:100FD000A906DF91CF91FF90EF90DF90CF90BF9067
:100FE000AF909F908F90089561E087E00E943A064D
:100FF00064E28EE70E943A0663E088E00E943A06C7
:1010000060E088E00E943A0665E087E00E943A06C8
:1010100062E085E00E943A0683E00E9434068093F5
:101020006B0384E00E94340680936A03089583E092
:101030000E94340680936B0384E00E943406809300
:101040006A0361E087E00E943A066AE070E080E0AF
:1010500090E00E9416190E94F40700000895CF92B4
:10106000DF92FF920F931F93CF93DF931F92CDB721
:10107000DEB7082F162F8EE399830E943A06F02ED2
:10108000C02E9981D92E8C2D8F19811738F4F60135
:1010900061916F018FE70E943A06F5CF64E085E029
:1010A0000E943A0683E00E94340680936B0384E03A
:1010B0000E94340680936A030E94F31860936603CB
:1010C00070936703809368039093690369E087E0F6
:1010D0000E943A0681E08093CD030F90DF91CF917B
:1010E0001F910F91FF90DF90CF9008950F931F9362
:1010F0000E942F088091CD03813099F40E94F3184B
:101100000091660310916703209168033091690391
:10111000601B710B820B930B603A764881409105FE
:1011200048F38091CD03813031F467EA71E087EDB7
:1011300093E00E94FB1B1F910F9108950F931F9343
:101140008091CD03823021F41092CD0381E020C044
:101150008091CD038130D9F40E94F3180091660389
:10116000109167032091680330916903601B710B34
:10117000820B930B613A76488140910540F061E023
:1011800087E00E943A061092CD0382E001C080E021
:101190001F910F910895CF93DF93EC014AE050E047
:1011A0006D2F70E087ED93E00E94C01C6EE287ED2A
:1011B00093E00E94CD1BBE0184E0769567958A95E9
:1011C000E1F76F7077274AE050E087ED93E00E94E7
:1011D000C01C6EE287ED93E00E94CD1BBE016F70D4
:1011E00077274AE050E087ED93E00E94C01CDF9132
:1011F000CF910895CF93C82F0E94F31860932A03CC
:1012000070932B0380932C0390932D03C0933F0383
:10121000CC2329F040E051EE60E070E004C040E8EB
:1012200055E260E070E089E294E00E940F1ECF91E9
:10123000089590912E03492F4F7050E0BA016F5FCF
:101240007F4F292F30E0E4E035952795EA95E1F7C7
:101250006217730759F0FA01E15DFC4F808381E06A
:10126000890F8F70907F892B80932E0308956EE7EE
:1012700070E089E294E00E94C90108951F920F92E4
:101280000FB60F9211241F932F933F934F935F93A9
:101290006F937F938F939F93AF93BF93CF93DF937E
:1012A000EF93FF93C0918600D09187008091E9026F
:1012B0009091EA0220910B03211155C09E01281B39
:1012C000390B8091B7039091B803A091B903B09105
:1012D000BA0385FD02C036952795253C49E03407C1
:1012E000B8F140910A0150E060E070E01CE1B69571
:1012F000A795979587951A95D1F70097A105B10500
:1013000021F481E090E0A0E0B0E084179507A60703
:10131000B707D8F480910A018F3FB9F040E080917F
:101320000A01481780F4842F90E0880F991FFC0170
:10133000E551FD4F20813181FC01E55FFE4F318396
:1013400020834F5FECCF10920C0310920A010BC068
:101350002D3B82E0380720F080910A018031D8F0DF
:101360008FEF80930A01D093EA02C093E902FF91C4
:10137000EF91DF91CF91BF91AF919F918F917F912D
:101380006F915F914F913F912F911F910F900FBEE1
:101390000F901F90189510910A0181E0810F8093A2
:1013A0000A01C9010E947805E12FF0E0EE0FFF1F4E
:1013B000E551FD4F91838083D6CF83E080938000F9
:1013C0008AE9809381008091B70386FD05C08091F2
:1013D00081008064809381008FEF9FEF909389005C
:1013E0008093880080916F00806280936F000895E1
:1013F0006F3018F086958058089589E0689F802D99
:1014000011240895A0E0B0E0E8E0FAE00C94EE23A7
:10141000C82F0E94F31800919A0210919B0220910C
:101420009C0230919D026B017C01C01AD10AE20A34
:10143000F30A9701860149E8C41643E1D406E104A2
:10144000F10410F010929E0260939A0270939B0236
:1014500080939C0290939D0220910B038FEF820F4B
:101460008230D8F5E0919E02EE2309F44EC1E130BE
:1014700011F482E0B8C1E03108F034C181E08E0F90
:1014800080939E02F0E0E551FD4FC083803109F06A
:10149000ACC1EDEEF2E0213029F4A181A695A6952C
:1014A000808108C080819181A92FA695A695A695D7
:1014B00096958795A03148F4B0E090E0AA0FBB1F45
:1014C000A55FBE4F11969C938E9310920C0332969B
:1014D00082E0EB3FF807F9F688C1233009F005C137
:1014E000E0919E02E11104C0CF3009F07EC10DC130
:1014F000E83148F481E08E0F80939E02F0E0E651DF
:10150000FD4FC08372C1E83109F0ECC0C111EAC0DF
:1015100040E050E0ABE0CA01B3E0880F991FBA95F4
:10152000E1F7A49F9001A59F300D1124F901E55129
:10153000FD4F6081E1817E2F777075956795FC0185
:10154000EE0FFF1FE55FFE4F71836083F901E451E9
:10155000FD4FB081B695B695B695E181FE2FF29517
:10156000FF0FF07E6F2F6B2BE695E695E6957E2FAD
:10157000777075956795FC01EE0FFF1FE35FFE4FD7
:1015800071836083F901E351FD4FB081B295B69547
:10159000B695B370C181DC2FDD0FDD0F6D2F6B2B86
:1015A000C295C695C695C370E281E170EE0FEE0F4D
:1015B0007E2F7C2B75956795FC01EE0FFF1FE15F79
:1015C000FE4F71836083F901E151FD4FB081B69503
:1015D000E181FE2FF795FF27F7956F2F6B2BE6958F
:1015E0007E2F777075956795FC01EE0FFF1FEF5EFC
:1015F000FE4F71836083F901E051FD4FB081B295D8
:10160000BF70E181FE2FF295F07F6F2F6B2BE2957B
:10161000EF707E2F777075956795FC01EE0FFF1FB9
:10162000ED5EFE4F71836083F901EF50FD4FB08195
:10163000BB1FBB27BB1FC181DC2FDD0F6D2F6B2BA9
:10164000CC1FCC27CC1FE281E370EE0F7E2F7C2BCA
:1016500075956795FC01EE0FFF1FEB5EFE4F7183E2
:101660006083F901ED50FD4FB081B695B695E181EB
:10167000FE2FF295FF0FFF0FF07C6F2F6B2BE6957F
:10168000E6957E2F777075956795FC01EE0FFF1F2D
:10169000E95EFE4F71836083F901EC50FD4F2081BC
:1016A0002295269527703181E32FEE0FEE0FEE0F76
:1016B0006E2F622B732F729576957770759567955F
:1016C000FC01EE0FFF1FE75EFE4F718360834F5FEB
:1016D0005F4F4230510509F01ECF8091010383FF17
:1016E00010920C0310929E0280C0243009F07DC03D
:1016F00060919E0261110BC0C83AB1F410926D0363
:1017000010926C0388EA0E94650281E06CC061302F
:1017100019F4C093990204C0623031F4C093980266
:101720008C2F0E9465025AC0E09198022E2F30E063
:10173000220F331F462F50E0C901029684179507E8
:101740003CF0633268F7FA01E851FD4FC083E8CFFF
:101750002D5F3F4F8C2F90E060916C0370916D0373
:101760004217530749F4982F882786279727909385
:101770006D0380936C0332C06817790769F5809117
:101780009902813049F5E13118F080E180939802A7
:10179000F0909802CCEED2E000E010E00F15D0F40B
:1017A000FE013197808190E0982F88272881822B35
:1017B00063E0969587956A95E1F70E947805F801B0
:1017C000EE0FFF1FE55FFE4F918380830F5F1F4F7A
:1017D0002296E4CF10920C0310929E0280919E02FA
:1017E000882319F08F5F80939E02CDB7DEB7E8E0C3
:1017F0000C940A24E82FF0E0EE54FC4FE185E03130
:1018000058F4F894F0E0EE0FFF1FE55FFE4F2081E3
:1018100031817894C9010895E03121F0E13169F412
:1018200083E001C082E00E94371A892B19F084EF0F
:1018300093E008958CE090E0089580E092E00895B0
:10184000A2E2B0E0E6E2FCE00C94E4239E012F5F0C
:101850003F4F80E1D9011D928A95E9F763EB71E072
:1018600087ED93E029A33AA30E94FB1B0E9417086F
:101870001D8A1E8A1F8A188E312C212C00E0812C93
:10188000912C540170EC472E7DE9572E78E5672E98
:1018900075E3772EE0E5CE2EE3ECDE2EE12CF12C85
:1018A00084EF91E0A0E0B0E08D8F9E8FAF8FB8A362
:1018B00080EC97EFAAEBB7E3898F9A8FAB8FBC8F41
:1018C00080EC9DE9A8E5B5E3898B9A8BAB8BBC8B4B
:1018D00087ED93E00E94601A892B09F4E1C087ED3F
:1018E00093E00E94841A9C0133272C32310509F4BD
:1018F00042C0ACF42332310509F0ABC019821A8220
:101900001B821C821D821E821F82188619861A86DF
:101910001B861C861D861E861F86188A60C024347E
:10192000310529F02335310509F4B2C092C064E4D1
:1019300087ED93E00E94CD1B2AE030E040EC5DE9AA
:1019400068E575E387ED93E00E945B1C6CE287ED30
:1019500093E00E94CD1B2AE030E040EC57EF6AEBA9
:1019600077E387ED93E00E945B1C6CE287ED93E0E8
:101970000E940D1CADCF0F5F043009F0A9CF298163
:101980003A814B815C81A8EEB3E00E946C23698BA5
:101990007A8B8B8B9C8B2D813E814F8158850E9449
:1019A0006C23698F7A8F8B8F9C8F29853A854B8525
:1019B0005C852D8F3E8F4F8F58A32D853E854F859B
:1019C00058890E946C236B017C0160323EE47307EE
:1019D0008105910530F462E38CE10E943A0600E053
:1019E00077CF603345E774078105910510F462E213
:1019F000F3CF60345CE975078105910510F466E268
:101A0000EBCF80E5C81683ECD806E104F10410F4AE
:101A100062E1E2CF90E6C9169AEED906E104F1043C
:101A200010F465E1D9CFA0E7CA16A1E1DA06A1E07A
:101A3000EA06F10410F461E0CFCFB0EACB16B6E8C5
:101A4000DB06B1E0EB06F10410F463E0C5CF65E01E
:101A5000C3CF10ED180F1A3008F03ACFE1E0F0E0F4
:101A6000EC0FFD1F24E0029FE00DF11D11242081E9
:101A7000318142815381AAE0B0E00E946C23610F62
:101A8000711D811D911D608371838283938320CF9B
:101A900049885A886B887C88812C912C540118CFF6
:101AA00081149104A104B10489F4C301B2010E941C
:101AB000A90661E070E080E090E00E9416191D8A9E
:101AC0001E8A1F8A188E312C22242A948D8D9E8D79
:101AD000AF8DB8A188169906AA06BB06D0F40E945D
:101AE00063062D893E894F89588D280F311D411D70
:101AF000511D2D8B3E8B4F8B588F381608F4382E86
:101B0000821508F4282E3FEF831A930AA30AB30A1A
:101B100056C0C301B20128EE33E040E050E00E941D
:101B2000A323BA01A9012AE030E087ED93E00E94E7
:101B3000A91C6CE287ED93E00E94CD1B4AE050E0C7
:101B4000632D87ED93E00E94B81C6CE287ED93E073
:101B50000E94CD1B6D897E898F89988DA501940186
:101B60000E94A323BA01A9012AE030E087ED93E0A7
:101B70000E94A91C6CE287ED93E00E94CD1B4AE015
:101B800050E0622D87ED93E00E94B81C6CE287ED77
:101B900093E00E940D1C4C0C5D1C6E1C7F1C898DFB
:101BA0009A8DAB8DBC8D84159505A605B70520F4DF
:101BB00049885A886B887C88812C912C540129890A
:101BC0003A894B895C89283E33404105510509F02B
:101BD0007FCEA296E2E10C940024ACE1B0E0E3EF0A
:101BE000FDE00C94EE230E94F3186B017C0181E070
:101BF0000E94190714E703E0198361E0CE01019602
:101C00000E9476080093CD030E94F4076AEF70E00B
:101C100080E090E00E9416198091CD03833089F412
:101C200087ED93E00E94601A892B59F40E94F31803
:101C30006C197D098E099F096038734C894C91405D
:101C4000D8F28091CD03833009F44FC08FE70E9412
:101C500012060E9425068983843511F083E05CC05A
:101C60000E94250610924003809341030E9425069E
:101C70002091400330914103280F311D30934103DF
:101C8000209340030E942506809342030E9425066C
:101C900080934303813110F7F12C0F2D10E08091D8
:101CA000430390E0880F991F0817190740F40E941A
:101CB0002506F801EC5BFC4F8083F394EECF80E7C0
:101CC000898361E0CE0101960E94760883E08093CB
:101CD000CD030E94F40762E370E080E090E00E9490
:101CE00016198091CD03833011F482E015C08FE77F
:101CF0000E9412060E9425068983803509F0AECF26
:101D000007E913E00E942506F80181938F01F3E0B3
:101D1000023B1F07B9F781E06C96E8E00C940A24B7
:101D2000CF93C82F682F87ED93E00E94D11A90912E
:101D300064039C2790936403CF910895A1E0B0E0E1
:101D4000E4EAFEE00C94F42399830E94900E9981BA
:101D5000892F0E94900E2196E2E00C9410241F938C
:101D6000CF93DF93182FEB011092640365EB87ED9F
:101D700093E00E94D11A62E687ED93E00E94D11AA7
:101D8000812F0E94900ECE010E949E0EDF91CF9176
:101D90001F9108956091640387ED93E00E94D11A2A
:101DA0000895A1E2B0E0E7EDFEE00C94F0237B01A2
:101DB0008A018B3009F42EC108F03FC0853009F448
:101DC0009BC010F5823009F47EC058F4813009F0D0
:101DD00030C269E270E081E00E94AF0E0EE613E0CF
:101DE00068C0833009F480C0843009F022C261E009
:101DF00070E084E00E94AF0E81E00E94900E0E948D
:101E0000CA0E0E94200C1FC2883009F49BC070F4D7
:101E1000863009F48DC0873009F00BC261E070E0B4
:101E200087E00E94AF0E8091420309C2893009F415
:101E300091C08A3009F4C3C0FCC1893609F469C174
:101E400078F4863609F41AC120F4853609F402C103
:101E5000F0C1873609F426C1883609F42BC1E9C1DF
:101E60008C3609F49FC190F48A3609F45CC18B3634
:101E700009F0DFC161E070E08BE60E94AF0EF8016F
:101E800080810E949F030E947904BEC18D3609F4AF
:101E9000BDC1873C09F0CDC161E070E087EC0E94D4
:101EA000AF0E81E00E94900E0E94CA0E1092650350
:101EB000CAC1F80181918F010E94900EF3E00739A9
:101EC0001F07B9F7BEC16BE170E082E00E94AF0E60
:101ED00007E913E0F80181918F010E94900EF3E071
:101EE000023B1F07B9F7ADC161E070E083E00E94DB
:101EF000AF0E0E94ED0DA3C16091430370E0660F29
:101F0000771F85E00E94AF0E04E413E08091430345
:101F100090E0880F991F98012454334028173907FF
:101F200008F08FC1F80181918F010E94900EEECFD1
:101F300062E070E086E00E94AF0E84E793E00E94CA
:101F40009E0E7FC161E070E088E00E94AF0E80913C
:101F5000CB0375C186E6898361E0CE0101960E94BC
:101F600076080E94F40783E08093CD0368EC70E06C
:101F700080E090E00E9416198091CD038430D9F45E
:101F80008FE70E9412060E9425068983863469F431
:101F900060E270E089E00E94AF0E10E20E94250628
:101FA0000E94900E1150D1F74CC161E070E089E0C1
:101FB0000E94AF0E29C161E070E089E03DC169E196
:101FC00070E08AE00E94AF0E82E08093B20320911D
:101FD000CC038091B7039091B803A091B903B0915D
:101FE000BA03222311F0806801C08F778093B70372
:101FF0009093B803A093B903B093BA0302EB13E034
:10200000F80181918F010E94900EF3E00B3C1F07B5
:10201000B9F717C161E270E08BE00E94AF0E8091CA
:102020000C038F3F39F080910C0391E0980F90934F
:102030000C0302C080910C030E94900E10E0812FCF
:102040000E94FA0B0E94A3050E949E0E1F5F103192
:10205000B1F7F7C061E070E085E60E94AF0E89E25B
:10206000E816F10409F0EAC0D801EEE6F3E08D913C
:10207000819383E0E739F807D1F7C6C061E070E0EB
:1020800086E60E94AF0EEBE1EE16F10409F0D6C031
:10209000D801E7E9F3E08D91819383E0E23BF80713
:1020A000D1F7B2C061E070E087E60E94AF0E0E94F7
:1020B0007004AAC061E070E088E60E94AF0E85E778
:1020C00089838BE1E7E9F3E0DE01129601900D923E
:1020D0008A95E1F76CE1CE0101960E9476080E9494
:1020E000F40783E08093CD0360E273E080E090E04A
:1020F0000E9416198091CD03843009F09FC08FE7AC
:102100000E9412060E9425068983853509F096C033
:102110007BC061E070E089E60E94AF0E0E94480338
:102120000E94B70371C061E070E08AE60E94AF0EC2
:1021300089E6898361E0CE0101960E9476080E94BB
:10214000F40783E08093CD0360E273E080E090E0E9
:102150000E9416198091CD03843009F06FC08FE77B
:102160000E9412060E94250689838E010E5F1F4F72
:102170007E01EDE1EE0EF11C0E942506F80181932F
:102180008F01EE15FF05C1F78BE1FE013296A7E93D
:10219000B3E001900D928A95E1F78981893409F0C5
:1021A0004DC032C061E070E08CE60E94AF0EF0E2FC
:1021B000EF16F10461F487E6898380E2F801DE011D
:1021C000129601900D928A95E1F761E203C087E4CF
:1021D000898361E0CE0101960E9476080E94F4078F
:1021E00083E08093CD036CE474E080E090E00E9493
:1021F00016198091CD03843009F58FE70E941206ED
:102200000E9425068734D1F481E019C061E070E0B6
:102210008DE60E94AF0E89E1E816F10479F4D80149
:10222000E2EBF3E08D91819383E0EB3CF807D1F78B
:10223000EBCF61E070E08AEC0E94AF0E80E00E947C
:10224000900E0E94CA0EA196E6E00C940C24A0E029
:10225000B0E0EDE2F1E10C94EE23CCE2D2E014E642
:1022600006E035E0F32E44E0E42E53E0D52E62E0A4
:10227000C62E87ED93E00E94601A892B09F49BC05B
:1022800087ED93E00E94841A282F80939702409153
:10229000960250E04730510560F7FA01EA5AFF4FC5
:1022A0000C941B24853B29F781E080939602E1CFB3
:1022B000823609F07DC0C0929602DBCF80939502F2
:1022C00080939402D0929602D4CF9C01332730930E
:1022D00093022093920290919402982790939402F3
:1022E000E0929602C6CF382F222740919202509159
:1022F0009302242B352B30939302209392029091DA
:102300009402982790939402F09296022536310514
:1023100008F4AFCF61E070E08CEC0E94AF0E81E07A
:102320000E94900E0E94CA0E43C0209190023091EC
:102330009102F901E45DFD4F80839091940298270A
:1023400090939402C9010196909391028093900218
:1023500020919202309193028217930708F489CF5B
:102360000093960286CF8091940282130BC06091F5
:102370009002709191024CE252E0809195020E948D
:10238000D10E0DC062E070E08BEC0E94AF0E809128
:1023900095020E94900E809164030E94900EFE01AF
:1023A000812F11928A95E9F7109291021092900272
:1023B000109296025ECFCDB7DEB7E8E00C940A2407
:1023C00081E08093650380916503882349F087ED60
:1023D00093E00E94601A892BB1F30E942711F3CF7A
:1023E0000895AAE2B0E0E7EFF1E10C94EC230E943B
:1023F000E7186B017C0181E00E94190787ED93E0EB
:102400000E94601A892B29F087ED93E00E94841ABC
:10241000F5CF5F9811E072E6B72EE9E2AE2E03E049
:102420000E94E7186C197D098E099F09693C7105A6
:1024300081059105D0F11123C1F10E94E7186B01CC
:102440007C01469A80ED97E00E94EC01B982EEE6AD
:10245000F3E0DE0112968A2D01900D928A95E1F744
:102460006AE2CE0101960E947608469880E090E0EC
:102470000E94EC010093CD030E94F40762E370E038
:1024800080E090E00E9416198091CD03843061F4C1
:102490000093CD038FE70E9412060E94250611E0EB
:1024A000823419F410E001C011E082E10E94371A71
:1024B000892B81F411E00EC05F9A469A87ED93E074
:1024C0000E94841A8D309105A9F05CF40A9791F06E
:1024D0005F98469887ED93E00E94601A892B61F718
:1024E0009FCF8332910569F08234910589F70E946C
:1024F000E011EECF66ED70E087ED93E00E94E91BFE
:10250000E7CF0E94200CE4CF8F929F92AF92BF92B0
:10251000CF92DF92EF92FF921F93CF93DF9382E1EE
:102520000E94371A892B09F078C068EC70E080E0CF
:1025300090E00E94161980E090E00E94EC010E9459
:10254000E7184B015C016B017C0180ECC80E82E155
:10255000D81EE11CF11C0E94E7186C157D058E0544
:102560009F0530F482E10E94371A892BA1F353C0F2
:1025700082E10E94371A892B09F04DC080ED97E067
:102580000E94EC010E94E7186B017C01D0E0C1E0E1
:1025900088E4880E86E2981EA11CB11C11E082E13D
:1025A0000E94371A892B21F58C149D04AE04BF04B8
:1025B00030F480ED97E00E94EC01D1E0F0CF0E9472
:1025C000E7186C197D098E099F09693C7105810521
:1025D000910528F30E94E7186B017C01C12719F0CF
:1025E00080ED97E002C080E090E00E94EC01D7CF40
:1025F00080E090E00E94EC01DD2349F08091CB0364
:102600008F5F83700E949F030E94790406C00E941E
:10261000D7030E9470040E94F111DF91CF911F91A6
:10262000FF90EF90DF90CF90BF90AF909F908F90F2
:102630000895CF92DF92EF92FF9280E00E944902CC
:102640000E940D0261E086E00E94CB1961E085E006
:102650000E94CB1960E082E10E94CB1960E084E027
:102660000E94CB1961E084E00E94041A0E94E001FC
:1026700060E070E087ED93E00E94561B0E94920399
:102680000E9479040E94DD098FEF80930C030E9461
:10269000190278940E94E7186B017C0180910C0369
:1026A0008F3F59F40E94E7186C197D098E099F0924
:1026B000603D77408105910588F380ED97E00E94A9
:1026C000EC0161E082E10E94041A5F9A87ED93E0D9
:1026D0000E94601A892B29F087ED93E00E94841AEA
:1026E000F5CF60EC71E087ED93E00E94CA1B84E7B0
:1026F00093E00E94CB0867ED71E087ED93E00E94C4
:10270000CA1B4AE050E066E070E087ED93E00E946B
:10271000911C62E370E080E090E00E94161987ED62
:1027200093E00E94601A04970CF187ED93E00E94F9
:10273000841A82349105D1F487ED93E00E94841AC3
:102740008E34910599F487ED93E00E94841A8434C5
:10275000910561F487ED93E00E94841A819731F42A
:1027600080E090E00E94EC010E94F11140916F0323
:10277000509170036091710370917203DB01CA0183
:102780000197A109B1090497A105B10568F4409327
:102790000B03433029F440EA56E861E070E004C0DE
:1027A00040E052EC61E070E089E294E00E940F1E8C
:1027B0000E9484125F9880E090E00E94EC010E94E9
:1027C000DD09109227038091B70383FF11C0809128
:1027D0008303882351F080918A03882331F080910C
:1027E0009103882311F087E001C085E080932703DF
:1027F00080E00E941907809128030E944D060E94E4
:10280000F4071092A1021092A00210929F02F12CE4
:102810008091CB038F15B0F062E370E080E090E030
:102820000E94161980ED97E00E94EC0162E370E0CF
:1028300080E090E00E94161980E090E00E94EC0198
:10284000F394E6CF8091960384FF08C0982F987187
:1028500081E0983109F080E00E94FA088FE00E9440
:102860004902FF90EF90DF90CF900895EF92FF9292
:102870000F931F93CF93DF938C016EE770E089E293
:1028800094E00E94C901E801F12CF0E2EF2E8E01E4
:1028900088818D57823048F46DE770E089E294E0DA
:1028A0000E94C90188818E2588832196F801608164
:1028B00089E294E00E94211DF394F9E0FF12E7CF32
:1028C0006EE770E089E294E00E94C901CDB7DEB7FF
:1028D000E6E00C940C24A9E0B0E0E1E7F4E10C940C
:1028E000F4239091290391110EC09EEF99838A835E
:1028F0006B8350E0559547954C832D831986188638
:102900001F821E822EC040912E03842F90E0B4E0DF
:1029100095958795BA95E1F7242F2F7030E08217AF
:10292000930719F18DEF89831B82FE01349650E0E5
:10293000842F90E0A4E095958795AA95E1F7242F40
:102940002F7030E08217930749F0DC01A15DBC4F86
:102950008C918193405F5F5F563051F740932E0317
:102960005A83CE0101960E9436148091290390E08B
:10297000019666E070E00E948F23809329032996D8
:10298000E2E00C941024A0E0B0E0E9ECF4E10C9457
:10299000ED236C016EE770E089E294E00E94C901CA
:1029A0008601E12CF12CC0E0D0E030E2B32EF8013A
:1029B000608183E8860F823078F46DE770E089E209
:1029C00094E00E94C901F80160816B2570E089E202
:1029D00094E00E94C90104C089E294E00E94211D94
:1029E000E114F10459F0F80180819E01280F311D96
:1029F000C901C92FDD27C80FD91FDD273FEFE31A13
:102A0000F30A89E0E816F10459F028E0E216F1042F
:102A100021F48C2F8095F60180870F5F1F4FC7CF61
:102A2000CDB7DEB7E9E00C940924A9E0B0E0EBE112
:102A3000F5E10C94F423E82F362F8091290390E0E0
:102A4000019664E270E00E948F238093290358E985
:102A5000598350E15A83813089F048F08230B9F0CF
:102A60008330D9F48B8381EF8C833D8319C085E05B
:102A70008B8381EF8C832F5F2D8312C08B8381EF3B
:102A80008C8384E6489FA00111245D8309C084E003
:102A90008B8381EF8C83ED8303C00E94370904C0D0
:102AA000CE0101960E94C3142996E2E00C941024F2
:102AB000A2E0B0E0EEE5F5E10C94E923182F762EC4
:102AC0002A8349830E94F3186B017C0180913F03A4
:102AD00080902A0390902B03A0902C03B0902D039C
:102AE0002A8149818823C1F0D701C6018819990933
:102AF000AA09BB094C015D0191EE89169EE2990677
:102B0000A104B10420F1241708F4422F202F672DCF
:102B1000812F0E94151513C0D701C6018819990984
:102B2000AA09BB094C015D0191E3891695E7990655
:102B3000A104B10460F0672D812F0E946B14C09234
:102B40002A03D0922B03E0922C03F0922D032296BD
:102B5000EDE00C940524A2E2B0E0E1EBF5E10C9489
:102B6000EA238CE00E94340681110DC06FED71E004
:102B700087ED93E00E94FB1B5F9A80E00E9419079B
:102B80000E94F4075F9889E294E00E94C71C892B99
:102B900001F189E294E00E94F41C90910B039923C7
:102BA00019F00E94020AEFCF4091A00250E09A0172
:102BB0002F5F3F4F2F7133276091A10270E02617DE
:102BC000370709F3FA01E555FD4F80832093A002F2
:102BD000DACF80910B03811106C08091CD03843040
:102BE00009F094C00DC087ED93E00E94601A892B14
:102BF000A1F387ED93E00E94841A0E94020AF3CFAA
:102C00000E94F318611571058105910549F06093E3
:102C1000190370931A0380931B0390931C030CC039
:102C200081E090E0A0E0B0E08093190390931A0354
:102C3000A0931B03B0931C0380910F03909110038A
:102C400081609093100380930F0383E08093CD0302
:102C50008FE70E9412060BEC12E00E942506F80195
:102C600081938F01F2E0043D1F07B9F72091D40250
:102C70008091CB02982F922796FF3BC090E4922739
:102C80009093D402982F98739833F1F410E0212F89
:102C900030E08091CB02877090E0821793074CF16F
:102CA0001F5F20919603812F90E0FC01E553FD4FBB
:102CB00024FF04C080810E941909E9CF608189E264
:102CC00094E00E94211DE3CF8F7399F48091CC0290
:102CD000809318038091CD02809316038091CE02D9
:102CE000809315038091D10290E090930E0380931E
:102CF0000D0380919F02813019F482E080939F023E
:102D000080919F02833011F410929F020E94F31869
:102D10006B017C018091110390911203A091130328
:102D2000B09114030097A105B105C9F0A701960160
:102D3000281B390B4A0B5B0BDA01C901883B9B400E
:102D4000A105B10560F00E946306809317031092FD
:102D50001103109212031092130310921403809126
:102D60001D0390911E03A0911F03B0912003460103
:102D70005701881A990AAA0ABB0A8EE693E00E94B4
:102D80008E0486169706A806B90608F4A4C0C09259
:102D90001D03D0921E03E0921F03F09220030E94B5
:102DA000C00180910C038830A0F08091B70390910E
:102DB000B803A091B903B091BA036CE1B695A79599
:102DC000979587956A95D1F7892B8A2B8B2B09F0DC
:102DD000A7C180910C038F5F80930C03809119032E
:102DE00090911A03A0911B03B0911C030097A105B9
:102DF000B105F1F0C81AD90AEA0AFB0A8EE693E097
:102E00000E948E046C157D058E059F0508F002C199
:102E10008091B70384FD04C080ED97E00E94EC012F
:102E20001092190310921A0310921B0310921C03A4
:102E30009091D402907C9093D4025091A002809102
:102E4000A10220919F02581709F401C1223009F014
:102E5000FEC090589093D402E0919603E770F0E0A2
:102E6000E251FE4F6081693008F0D9C0615040E006
:102E70004613D7C08093A10287E3840F9091D402B8
:102E8000892B8093D4024093A20283E080939F0217
:102E9000469A9091270391112DC1809128030E9499
:102EA0004D06E0919603E770F0E0E251FE4F60813D
:102EB00084ED92E00E942F08E0912803EF5FE093F9
:102EC0002803E83109F429C1F0E0E259FC4F878575
:102ED000882309F422C10E949E08813069F58091FF
:102EE0009603887149F180910F0390911003880F28
:102EF000991F9093100380930F0383E08093CD0379
:102F00000E94F4070E94F318609311037093120358
:102F10008093130390931403672B682B692B61F440
:102F200081E090E0A0E0B0E0809311039093120361
:102F3000A0931303B09314038091960384FF1FC0E2
:102F400080910F03909110038E7F0E94C405182F6B
:102F500060910D03809118030E94F809482F612F9A
:102F60008091170349A30E94F8090091CB03282FF1
:102F700049A160911503809116030E945815469847
:102F8000809125038130C1F018F08230B1F1D1C0B9
:102F900082E10E94371A892B09F0CBC081E080932F
:102FA00025030E94E7186093210370932203809306
:102FB000230390932403BDC082E10E94371A892B1A
:102FC00031F50E94E718C0902103D0902203E090D1
:102FD0002303F09024036C197D098E099F09693E33
:102FE00073408105910508F4A4C082E08093250315
:102FF00080ED97E00E94EC019CC082E10E94371AAC
:10300000892B09F496C080E090E00E94EC011092B8
:1030100025038FC080E090E00E94EC0109CF68E0BA
:1030200026CF851709F426CF4F5F242F30E090E09C
:10303000F901EC52FD4FDC01A555BD4F7C91708329
:10304000F901EE55FD4F708301968F7111CF243039
:10305000B1F42091A20283EA92E0A5EDB2E0FC0176
:103060003E2F381B321718F431913D93F9CF87E387
:10307000820F9091D402892B8093D40206CF809145
:103080002503823069F491609093D4025F9A5BEBE0
:10309000E52E53E0F52E8E010F5F1F4FB80110C0D3
:1030A0005F9880919F02811103C081E080939F020D
:1030B00080919F02833059F784E080939F02E7CF8D
:1030C000F70181917F0169A37AA30E94FA0BF801AD
:1030D000819391938F0169A17AA1FBECEF16F3E044
:1030E000FF0671F78091960345ED52E087700E94CC
:1030F0001305CECE80917B03882309F4CECE209198
:10310000260331E0320F30932603291303C01092B7
:10311000260381500E941407C0CE10922803DBCEF4
:1031200080910C03883009F45F9A89E080930C0346
:10313000D2CEA296ECE00C9406241F920F920FB60A
:103140000F9211242F933F938F939F93AF93BF932D
:103150008091CF039091D003A091D103B091D2037D
:103160003091CE0323E0230F2D3720F40196A11DCB
:10317000B11D05C026E8230F0296A11DB11D2093A5
:10318000CE038093CF039093D003A093D103B09349
:10319000D2038091D3039091D403A091D503B09131
:1031A000D6030196A11DB11D8093D3039093D40340
:1031B000A093D503B093D603BF91AF919F918F9108
:1031C0003F912F910F900FBE0F901F9018952FB722
:1031D000F8946091CF037091D0038091D1039091C6
:1031E000D2032FBF08953FB7F8948091D3039091F5
:1031F000D403A091D503B091D60326B5A89B05C0F2
:103200002F3F19F00196A11DB11D3FBF6627782FF2
:10321000892F9A2F620F711D811D911D42E0660F4B
:10322000771F881F991F4A95D1F70895CF92DF9293
:10323000EF92FF92CF93DF936B017C010E94F31812
:10324000EB01C114D104E104F10479F00E94F318F8
:103250006C1B7D0B683E7340A0F381E0C81AD10857
:10326000E108F108C851DC4FECCFDF91CF91FF901E
:10327000EF90DF90CF900895789484B5826084BDFC
:1032800084B5816084BD85B5826085BD85B581606A
:1032900085BDEEE6F0E0808181608083E1E8F0E0CA
:1032A0001082808182608083808181608083E0E8F9
:1032B000F0E0808181608083E1E9F0E080818260DC
:1032C0008083808181608083E0E9F0E0808181609B
:1032D0008083E1ECF0E08081846080838081826083
:1032E0008083808181608083E3ECF0E08081816075
:1032F0008083E0ECF0E0808182608083E2ECF0E0AB
:10330000808181608083EAE7F0E08081846080834F
:1033100080818260808380818160808380818068F9
:103320008083089590E0FC013197EE30F10590F52F
:10333000E35AFF4F0C941B24809180008F7703C0C9
:10334000809180008F7D80938000089584B58F7771
:1033500002C084B58F7D84BD0895809190008F77E1
:1033600007C0809190008F7D03C080919000877F7F
:103370008093900008958091C0008F7703C0809162
:10338000C0008F7D8093C00008958091C200877F28
:103390008093C2000895CF93DF9390E0FC01E75E35
:1033A000FE4F2491FC01E95CFE4F8491882349F192
:1033B00090E0880F991FFC01EF58FE4FA591B49142
:1033C0008D599E4FFC01C591D4919FB7611108C0E2
:1033D000F8948C91209582238C93888182230AC053
:1033E000623051F4F8948C91322F309583238C9372
:1033F0008881822B888304C0F8948C91822B8C93D3
:103400009FBFDF91CF910895A1E0B0E0EAE0FAE13B
:103410000C94F223282F30E0F901E550FF4F8491FE
:10342000F901E75EFE4F1491F901E95CFE4F04914A
:103430000023C9F0882321F069830E9492196981D1
:10344000E02FF0E0EE0FFF1FED59FE4FA591B49174
:103450009FB7F8948C91611103C01095812301C02E
:10346000812B8C939FBF2196E4E00C940E24CF9384
:10347000DF93282F30E0F901E550FF4F8491F901E7
:10348000E75EFE4FD491F901E95CFE4FC491CC2375
:1034900091F081110E949219EC2FF0E0EE0FFF1FC6
:1034A000EB5AFE4FA591B4912C912D2381E090E031
:1034B00021F480E002C080E090E0DF91CF91089598
:1034C00080912504909126042091270430912804AE
:1034D000821B930B8F7399270895209125043091B7
:1034E000260480912704909128042817390749F071
:1034F000E0912704F0912804EB51FC4F808190E08B
:1035000008958FEF9FEF08952091250430912604B0
:10351000809127049091280428173907A9F0E09199
:103520002704F0912804EB51FC4F8081209127045F
:10353000309128042F5F3F4F2F7333273093280497
:103540002093270490E008958FEF9FEF0895CF9385
:10355000DF93C0912504D09126042196CF73DD27F7
:103560008091270490912804C817D90799F082E028
:103570000E94451F8F3F2FEF920761F0E0912504D5
:10358000F0912604EB51FC4F8083D0932604C09326
:103590002504DFCFDF91CF91089583E00E94902131
:1035A0000895A1E0B0E0E7EDFAE10C94F2238C017C
:1035B00069838091A401882359F041E050E0BE0165
:1035C0006F5F7F4F83E00E94781F181619063CF04A
:1035D00081E090E0F8019383828380E090E021967F
:1035E000E4E00C940E24FC0120812E5F208342E451
:1035F00050E06FE771E080E80E94F81F0895FC0139
:1036000081819081913A59F4813209F04BC047E0B1
:1036100050E06DE971E080E00E94F81F45C09132F2
:1036200009F040C0803239F467E070E08DE991E044
:103630000E943C2039C0823209F034C082818093DC
:10364000A40180919D0190919E01A0919F01B09154
:10365000A001803B9440A105B10531F58091A40102
:1036600080FD12C087E797E79093010880930008D8
:103670002BE088E190E00FB6F894A8958093600065
:103680000FBE2093600010C088E10FB6F8948093BD
:103690006000109260000FBEA89510920108109271
:1036A000000802C080E0089581E008950895109216
:1036B000DA031092D90388EE93E0A0E0B0E08093A3
:1036C000DB039093DC03A093DD03B093DE0380E083
:1036D00092E09093D8038093D7030895A0E0B0E0E0
:1036E000E4E7FBE10C94EE236C017A01EB01E60EBA
:1036F000F71E00E010E0CE15DF0561F06991D601FC
:10370000ED91FC910190F081E02DC6010995080F23
:10371000191FF1CFC801CDB7DEB7E8E00C940A2439
:103720006115710589F0DB010D900020E9F7AD010D
:1037300041505109461B570BDC01ED91FC91028071
:10374000F381E02D0995089580E090E00895EF92CF
:10375000FF920F931F93CF93DF938C01FB01C0E087
:10376000D0E064917F018FEFE81AF80A662361F0D8
:10377000D801ED91FC910190F081E02DC8010995EF
:10378000C80FD91FF701EDCFCE01CDB7DEB7E6E008
:103790000C940C240E94901B0895DC01ED91FC9187
:1037A0000190F081E02D099508950F931F93CF9319
:1037B000DF93EC016DE00E94CD1B8C016AE0CE012D
:1037C0000E94CD1B800F911FDF91CF911F910F9110
:1037D00008950F931F93CF93DF93EC010E94A71BD3
:1037E0008C01CE010E94D51B800F911FDF91CF91DC
:1037F0001F910F9108950F931F93CF93DF93EC01C7
:103800000E94901B8C01CE010E94D51B800F911F3E
:10381000DF91CF911F910F9108950F931F93CF9335
:10382000DF93EC010E94CD1B8C01CE010E94D51BC1
:10383000800F911FDF91CF911F910F910895A1E209
:10384000B0E0E5E2FCE10C94EA237C01C42EE52F14
:10385000CB01D22E19A221E02D1510F02AE0D22E94
:103860008E010F5D1F4F8D2C912CA12CB12C6C2D36
:103870007E2FA50194010E94A3238C2DD29E801936
:103880001124015011098A3010F4805D01C0895C57
:10389000F8018083211531054105510521F0C22E23
:1038A000E32FCA01E4CFB801C7010E94901BA19683
:1038B000ECE00C940624A0E0B0E0E1E6FCE10C941E
:1038C000EE23EC016A017B012115310541F4E88109
:1038D000F9810190F081E02D642F09951DC02A30F7
:1038E0003105A9F477FF12C06DE20E94CD1B8C0157
:1038F00044275527BA014C195D096E097F092AE052
:10390000CE010E941F1C800F911F06C02AE0B70144
:10391000A601CE010E941F1CCDB7DEB7E8E00C94D3
:103920000A240F931F93CF93DF93EC019A01AB010D
:10393000662757FD6095762F0E945B1C8C01CE0197
:103940000E94D51B800F911FDF91CF911F910F9186
:1039500008952115310549F4DC01ED91FC910190A8
:10396000F081E02D642F099508950E941F1C089591
:103970009A01462F50E060E070E00E94A91C089573
:103980009A01AB0160E070E00E94A91C0895FC015F
:1039900024853585F901E05CFF4F80819181F90133
:1039A000EE5BFF4F20813181821B930B8F73992730
:1039B0000895FC0184859585FC01E05CFF4F408102
:1039C0005181FC01EE5BFF4F20813181421753078B
:1039D00041F00190F081E02DE80FF91F808190E027
:1039E00008958FEF9FEF0895FC0184859585FC0174
:1039F000E05CFF4F40815181FC01EE5BFF4F208175
:103A000031814217530779F0A081B181A80FB91F06
:103A10008C91208131812F5F3F4F2F73332731836A
:103A2000208390E008958FEF9FEF0895FC0181A11E
:103A3000882329F0A489B5898C9186FFFBCF11A238
:103A40000895CF93DF93FC0126853785D901A05CCB
:103A5000BF4F8D919C91119701968F739927E90122
:103A6000CE5BDF4F4881598184179507D9F30D90BC
:103A7000BC91A02DA20FB31F6C93A685B785A05C47
:103A8000BF4F11969C938E93A689B7892C9181E0A4
:103A900090E0078C02C0880F991F0A94E2F7282B48
:103AA0002C9381E081A30488F589E02D80818064D6
:103AB000808381E090E0DF91CF91089508951F9277
:103AC0000F920FB60F9211242F933F934F938F9322
:103AD0009F93EF93FF938091C80082FD1CC040919B
:103AE000CE008091CF049091D00401968F739927D6
:103AF0002091D1043091D2048217930771F0E091A4
:103B0000CF04F091D004E157FB4F40839093D00451
:103B10008093CF0402C08091CE00FF91EF919F91DE
:103B20008F914F913F912F910F900FBE0F901F904B
:103B3000189589E294E00E94C71C892B11F00E941D
:103B40005E1D08951F920F920FB60F9211242F93AE
:103B50003F938F939F93EF93FF9320918B0430912A
:103B60008C0480918D0490918E042817390731F4CC
:103B70008091C9008F7D8093C90014C0E0918D04AD
:103B8000F0918E04E55BFB4F208180918D04909134
:103B90008E0401968F73992790938E0480938D04E1
:103BA0002093CE00FF91EF919F918F913F912F91A4
:103BB0000F900FBE0F901F901895A0E0B0E0E3EEBD
:103BC000FDE10C94EA23FC011382128288EE93E05B
:103BD000A0E0B0E084839583A683B78382E192E07E
:103BE000918380837587648757874687318B208BC5
:103BF000138B028BF58AE48AD78AC68AB18EA08E8F
:103C0000938E828E8F85848F8889858F8989868F10
:103C10008A89878F8B8980A3ECE00C940624CF924D
:103C2000DF92EF92FF92CF93DF93EC016A017B0169
:103C3000411581EE580761057105F9F0EC89FD89A0
:103C400081E090E008A002C0880F991F0A94E2F773
:103C5000808360E079E08DE390E0A70196010E9407
:103C6000A3232150310941095109569547953795AC
:103C70002795211580E1380798F0EC89FD8910829D
:103C800060E874E88EE190E0A70196010E94A3230A
:103C90002150310941095109569547953795279586
:103CA000E889F9893083EA89FB89208319A2EE89A2
:103CB000FF89408181E090E09C010C8C02C0220FC2
:103CC000331F0A94E2F7422B4083EE89FF8940813B
:103CD0009C010D8C02C0220F331F0A94E2F7422B85
:103CE0004083EE89FF8940819C010E8C02C0220F27
:103CF000331F0A94E2F7422B4083EE89FF8920812B
:103D00000F8C02C0880F991F0A94E2F780958223D6
:103D10008083DF91CF91FF90EF90DF90CF90089557
:103D20008F929F92AF92BF92CF92DF92EF92FF92CB
:103D30000F931F9381E08F9385E08F9387E08F939C
:103D400083E08F9384E08F93EEEC8E2E912CFAEC2F
:103D5000AF2EB12CA9ECCA2ED12CB8ECEB2EF12C45
:103D60000CEC10E02DEC30E04BE454E06FE874E034
:103D700089E294E00E94DD1D0F900F900F900F904C
:103D80000F901F910F91FF90EF90DF90CF90BF9019
:103D9000AF909F908F9008950E943C1983ED94E01E
:103DA0000E949A210E941913C9E9DDE10E94AB1516
:103DB0002097E1F30E94991DF9CF615030F02091D6
:103DC000F100FC0120830196F8CF289884E68093C7
:103DD000DA0408952FB7FC012083F894677060938C
:103DE000E9000895A1E0B0E0E8EFFEE10C94F423CF
:103DF000682FCE0101960E94EA1E8091F2009981FF
:103E00009FBF2196E2E00C941024A2E0B0E0EBE02A
:103E1000FFE10C94F123F62E8A019091D9049923A5
:103E200011F057FF03C08FEF9FEF2BC0682FCE011B
:103E300001967A830E94EA1E8091F20090E0A80128
:103E40007A81801791070CF4AC01EF2DF72FF40E57
:103E500084E6FE1639F028988093DA049091F100F8
:103E60009193F7CF4115510521F08091F2008823FD
:103E700021F089818FBFCA0104C08BE68093E800DE
:103E8000F8CF2296E5E00C940D24A1E0B0E0EBE43D
:103E9000FFE10C94F42341E050E0BE016F5F7F4FDF
:103EA0000E94051F019719F4898190E002C08FEFED
:103EB0009FEF2196E2E00C941024A1E0B0E0E3E64D
:103EC000FFE10C94F423682FCE0101960E94EA1EB4
:103ED0009091E800892F807295FF04C09091F200C4
:103EE00080E4891B99819FBF2196E2E00C94102405
:103EF000A1E0B0E0EEE7FFE10C94E623582E7B0151
:103F0000A42E952E8091D904882369F0042F152FB3
:103F10008AEFB82E852D8072782E9AE3892E852D12
:103F20008074682E11C08FEF9FEF53C0852D0E94C3
:103F30005D1F482E81110CC0BA94A9F361E070E0B6
:103F400080E090E00E9416190115110579F737C03D
:103F5000282F30E0021713070CF4402EC42CD12C6C
:103F60000C191D09652DCE0101960E94EA1E7720CD
:103F700039F04A948FEF4816B1F01092F100F9CF62
:103F8000F701842D57FE07C0815058F0949190930B
:103F9000F1003196F9CF815020F091919093F1008A
:103FA000FACFEC0CFD1C8091E80085FF0FC00115D5
:103FB000110511F461100AC089818FBFC5CF5D98CA
:103FC00084E68093DB048A2D992D03C08092E8005B
:103FD000F3CF2196E0E10C9402241092E9001092B4
:103FE000D8041092D7049093D6048093D5040895F2
:103FF000CF93DF93FB0120E030E0DEEF241735079D
:10400000A1F187FF02C0C49101C0C081A091D70473
:10401000B091D8046091D5047091D604A617B70763
:10402000B4F49091E8009570E1F39091E80092FD6E
:104030001EC0C093F1006091D7047091D8046F5FE7
:104040007F4F6F737727672B11F4D093E80060914F
:10405000D7047091D8046F5F7F4F7093D80460933A
:10406000D7042F5F3F4F3196C9CFC90102C08FEFF0
:104070009FEFDF91CF910895A1E0B0E0E2E4F0E29C
:104080000C94F323162F2091E80022FFFCCF612F20
:1040900079830E94DD1E8BEF8093E800812F798168
:1040A000972F2196E3E00C940F24A1E0B0E0EBE51C
:1040B000F0E20C94F4231982CE0101960E94F31AC7
:1040C000CE0101960E943422898190E02196E2E09F
:1040D0000C9410241F920F920FB60F921124EF929E
:1040E000FF920F931F932F933F934F935F936F9381
:1040F0007F938F939F93AF93BF93EF93FF93CF9350
:10410000DF93CDB7DEB76297DEBFCDBF1092E90077
:104110008091E80083FFE7C068E0CE010A960E9424
:10412000DD1E82EF8093E8009A8597FF05C080919D
:10413000E80080FFFCCF03C08EEF8093E800892F5A
:10414000807609F0B5C08B85811105C01092F10011
:104150001092F100C1C0282F2D7F213009F4BCC07E
:10416000853049F48091E80080FFFCCF8C85806821
:104170008093E300B1C0863009F072C02D85E888D5
:10418000F988223071F580E090E02A8B0E94ED1FC3
:104190000E94552099E08E010F5F1F4FF801392FC3
:1041A00011923A95E9F799832A892A8391E09E83AF
:1041B00090E898879AEF99872091D7043091D80496
:1041C000275F3F4F3C832B838D83C7010E94ED1FE8
:1041D00049E050E0B80180E00E94F81F0E9455209D
:1041E0007BC0C7012A8B0E94ED1F2A89223241F42D
:1041F00082E290E00E944022892B09F06DC070C0DD
:10420000213069F488899989089711F42093D4049E
:104210008091D404882389F066EC71E016C02330C5
:1042200009F05EC08C85882359F0823061F08130BE
:1042300009F056C06AEE71E008C068ED71E005C093
:1042400064E272E002C062E072E06115710509F497
:1042500047C0FB01449150E080E80E94F81F3CC039
:10426000873009F43DC0883021F481E08093F1006B
:1042700033C0893089F5937099F5E2ECF1E081E083
:1042800021E096E38093E9002093EB003491309392
:10429000EC009093ED008F5F3196853099F78EE7B3
:1042A0008093EA001092EA008C858093D90414C0B0
:1042B000888999890E94ED1F8E85811105C0CE01E4
:1042C0000A960E94FF1A06C0823051F4CE010A9667
:1042D0000E946222882321F08EEF8093E80003C0C1
:1042E00081E28093EB0062960FB6F894DEBF0FBEBA
:1042F000CDBFDF91CF91FF91EF91BF91AF919F9192
:104300008F917F916F915F914F913F912F911F916D
:104310000F91FF90EF900F900FBE0F901F90189588
:104320008093E9008091F200882319F08AE380935A
:10433000E80008951092D90481E08093D70080EAC4
:104340008093D80082E189BD09B400FEFDCF61E011
:1043500070E080E090E00E94161980E98093D80018
:104360008CE08093E2001092E000559A209A089524
:104370001F920F920FB60F9211242F933F934F93DA
:104380005F936F937F938F939F93AF93BF93EF93BD
:10439000FF938091E1001092E10083FF0FC0109223
:1043A000E90091E09093EB001092EC0092E390937F
:1043B000ED001092D90498E09093F00082FF26C09F
:1043C00083E00E94902182E00E94F21E882321F067
:1043D00087ED93E00E94A71A8091DB04882339F0CF
:1043E0008091DB0481508093DB04882369F0809105
:1043F000DA04882359F08091DA0481508093DA043A
:10440000811104C0289A02C05D9AF1CFFF91EF910B
:10441000BF91AF919F918F917F916F915F914F91DC
:104420003F912F910F900FBE0F901F901895FF9204
:104430000F931F93CF93DF93EC01F62EE881F98160
:104440000480F581E02D09958C01E881F9810680D1
:10445000F781E02D6F2DCE010995C8019927CDB7C1
:10446000DEB7E5E00C940D24FC0120812F5F208352
:1044700049E150E068EA72E080E80E94F81F089580
:1044800045E650E061EC72E080E80E94F81F089574
:10449000A1E0B0E0EEE4F2E20C94F02389838B011A
:1044A0007A0141E050E0BE016F5F7F4F84E00E94DF
:1044B000781FA701B80184E40E94781F2196E6E0E6
:1044C0000C940C24FC0191818081813A31F481E0CB
:1044D000913091F0933089F411C0813271F49B30A6
:1044E00021F482818093A60105C09A3031F4828143
:1044F0008093A50181E00895089580E00895FC016E
:1045000010820895FC011382128222E232E031838C
:104510002083089548E050E082E00E9448220895F8
:10452000CF93DF93DC01683818F0E8E7E60F25C089
:10453000E62FF0E067FF11C0E058F10981E090E05C
:1045400001C0880FEA95EAF714969C911497982B6E
:1045500014969C931497E0E010C0E85DFD4FE49141
:10456000EE2309F440C0E7FF08C014968C9114971D
:10457000826014968C931497EF7716968C91169709
:104580008E1741F117968C9117978E1719F118967F
:104590008C9118978E17F1F019968C9119978E17A8
:1045A000C9F01A968C911A978E17A1F01B968C91D0
:1045B0001B978E1779F080E090E0ED01C80FD91FAE
:1045C0002E81211102C0EE8305C00196863091052F
:1045D000A1F709C0BD016C5F7F4FCD010E948A2207
:1045E00081E090E008C081E090E013969C938E9368
:1045F000129780E090E0DF91CF910895683818F02D
:10460000E8E7E60F25C0E62FF0E067FF12C0E058AC
:10461000F10921E030E001C0220FEA95EAF7209588
:10462000DC0114963C911497322314963C93E0E0FD
:104630000FC0E85DFD4FE491EE2329F1E7FF08C0CC
:10464000DC0114962C9114972D7F14962C93EF7700
:1046500020E030E0EE2351F0DC01A20FB31F1696EC
:104660004C9116974E1302C016961C922F5F3F4F27
:104670002630310579F7BC016C5F7F4F0E948A229A
:1046800081E090E0089580E090E00895FC011682BA
:10469000178210861186128613861482BC016C5F05
:1046A0007F4F0E948A22089588EE94E00E947F2224
:1046B0008CED94E00E9482220895A29FB001B39FE6
:1046C000C001A39F700D811D1124911DB29F700D1B
:1046D000811D1124911D08950E945D23A59F900DB9
:1046E000B49F900DA49F800D911D11240895B7FFD4
:1046F0000C946C230E946C23821B930B0895DB01A6
:104700008F939F930E946C23BF91AF91A29F800DC6
:10471000911DA39F900DB29F900D1124089597FBBA
:10472000072E16F4009407D077FD09D00E942124AB
:1047300007FC05D03EF4909581959F4F08957095A4
:1047400061957F4F0895A1E21A2EAA1BBB1BFD01A4
:104750000DC0AA1FBB1FEE1FFF1FA217B307E40760
:10476000F50720F0A21BB30BE40BF50B661F771FB8
:10477000881F991F1A9469F7609570958095909598
:104780009B01AC01BD01CF010895052E97FB1EF4DE
:1047900000940E94DC2357FD07D00E94A32307FC4E
:1047A00003D04EF40C94DC23509540953095219520
:1047B0003F4F4F4F5F4F089590958095709561954D
:1047C0007F4F8F4F9F4F08952F923F924F925F924E
:1047D0006F927F928F929F92AF92BF92CF92DF9211
:1047E000EF92FF920F931F93CF93DF93CDB7DEB776
:1047F000CA1BDB0B0FB6F894DEBF0FBECDBF09940A
:104800002A88398848885F846E847D848C849B8460
:10481000AA84B984C884DF80EE80FD800C811B816E
:10482000AA81B981CE0FD11D0FB6F894DEBF0FBE9D
:10483000CDBFED010895EE0FFF1F0590F491E02D1F
:104840000994AA1BBB1B51E107C0AA1FBB1FA617D7
:10485000B70710F0A61BB70B881F991F5A95A9F729
:1048600080959095BC01CD0108958F929F92AF9253
:10487000BF92CF92DF92EF92FF92CF93DF93EC0142
:10488000688179818A819B81611571058105910516
:1048900021F464E279ED8BE597E02DE133EF41E01F
:1048A00050E00E94C52349015A019B01AC01A7EACF
:1048B000B1E40E946C236B017C01ACEEB4EFA50166
:1048C00094010E947A23C60ED71EE81EF91EF7FE39
:1048D00006C081E0C81AD108E10880E8F80AC88259
:1048E000D982EA82FB82C701B6019F77DF91CF911F
:1048F000FF90EF90DF90CF90BF90AF909F908F9000
:1049000008950E943524089586E091E00E943524A0
:1049100008956093060170930701809308019093B6
:1049200009010895F999FECF92BD81BDF89A9927A2
:1049300080B50895262FF999FECF1FBA92BD81BD8B
:1049400020BD0FB6F894FA9AF99A0FBE0196089511
:04495000F894FFCF09
:104954000000E904200001000000FF000200020042
:104964000200020002000200020002000200020033
:10497400020002000200020002000280250000057D
:10498400400AA1204EA50020244EA52C2330C0129D
:1049940000001A400AA1204EA5001B1E27522C23FA
:1049A400308025000005400AA1204EA50020244E99
:1049B400A52C2330004B000006400AD0009D49007E
:1049C4007B289D492C233000E1000005400A450165
:1049D400D7DC03B81E0EBF00232E48E801008A402E
:1049E4000A6001555502AD1E20000023C800E100F5
:1049F4000000000000010154582074696D656F7552
:104A04007421007363616E6E6572206D6F6465005E
:104A14004F70656E4C52536E672054582073746106
:104A24007274696E672000206F6E20485720006DF5
:104A34006F64756C65206C6F636B65643F00000781
:104A44000B0C10111500160A132231290000000066
:104A5400D11A6E1B601A841A6D1ACD1AA71A000097
:104A64000000211D6E1BC71CF41CD91C161D000060
:0C4A7400000017226E1B9022FE22462339
:1070000055C000006EC000006CC000006AC00000E7
:1070100068C0000066C0000064C0000062C00000DC
:1070200060C000005EC00000F2C400005AC0000052
:1070300058C0000056C0000054C0000052C00000FC
:1070400050C0000078C000004CC000004AC00000E2
:1070500048C0000046C0000044C0000042C000001C
:1070600040C000003EC000003CC000003AC000002C
:1070700038C0000036C0000034C0000032C000003C
:1070800030C000002EC000002CC000002AC000004C
:1070900028C0000026C0000024C0000022C000005C
:1070A00020C000001EC000001CC0000011241FBE34
:1070B000CFEFDAE0DEBFCDBF11E0A0E0B1E0E2E368
:1070C000FFE702C005900D92A83AB107D9F711E089
:1070D000A8EAB1E001C01D92AE3BB107E1F78FD342
:1070E00026C78ECFF89410926F00109281001092F4
:1070F00085001092840081E085BF15BE47985D9A97
:10710000289A0C94000008952091B2013091B301A7
:107110002F5F3F4F3093B3012093B201932F37FF7E
:1071200003C08EEF831B982F990F921710F4479886
:107130000895479A08951F920F920FB60F92112447
:107140002F938F939F93EF93FF931092850010924C
:1071500084008091A8019091A901009741F00197C6
:107160009093A9018093A801892B09F45D9A8091DD
:10717000AA019091AB01009741F001979093AB0168
:107180008093AA01892B09F4289AE0E0F0E0859128
:1071900094918F5F9F4F49F08091AC019091AD0128
:1071A00001969093AD018093AC01FF91EF919F9177
:1071B0008F912F910F900FBE0F901F90189584E024
:1071C0008093E9000DC08091E8008B778093E80000
:1071D00003C08EB3882351F08091E80082FFF9CF7D
:1071E0008091E80085FFEFCF8091F1000895982FFE
:1071F00083E08093E9008091E80085FD0DC08091D7
:10720000E8008E778093E80003C08EB3882369F08E
:107210008091E80080FFF9CF9093F1005D9884E6BB
:1072200090E09093A9018093A80108954F925F92F6
:107230006F927F928F929F92AF92BF92CF92DF9286
:10724000EF92FF920F931F93CF93DF9384E080938D
:10725000E9008091E80082FF57C2289884E690E018
:107260009093AB018093AA01AADF182F853481F493
:107270008CE49DE19093AD018093AC0107B600FCD6
:10728000FDCFF999FECF81E180935700E89503C0C7
:10729000843519F494DF8DE00DC28C34E1F3803530
:1072A000D1F3843721F484E4A2DF80E003C2813685
:1072B00011F489E5FFC18134B1F481DF182F7FDF3C
:1072C00090E0880F991FAA2797FDA095BA2F312F1C
:1072D000330F20E0442737FD4095542F822B932B0A
:1072E000A42BB52BB8C1803711F483E5E3C18335F6
:1072F00049F4C0E0D1E089917ADF21E0C730D207BC
:10730000D1F7D9C1863521F481E371DF80E3D2C1A1
:10731000833731F487E86BDF85E969DF8EE1CAC125
:107320008536B9F4E0E0F0E093E085E09093570013
:10733000E89507B600FCFDCF80935700E89507B6A7
:1073400000FCFDCFE058FF4FA0E7E030FA0771F7EF
:10735000A2CF823739F4E1E0F0E089E08093570072
:107360008491A8C1863439F4E0E0F0E089E08093AC
:10737000570084919FC18E3439F4E3E0F0E089E056
:1073800080935700849196C1813539F4E2E0F0E0B2
:1073900089E08093570084918DC1823631F489E56C
:1073A00026DF80E024DF80E885C1823419F087364B
:1073B00009F0E5C01092AD011092AC0100DF082F7A
:1073C000FEDEF82EFCDE682E8554823008F071C196
:1073D000902F80E0CF2DD0E0C82BD92B10926F00DA
:1073E000173609F04BC081E180935700E895DD2402
:1073F000CC24C3943FC0E090AE01F090AF01009167
:10740000B0011091B101B6E46B16D9F4ED2DF0E0A6
:10741000EE29FF29E4918E2FEADEDD2081F082E063
:1074200090E0A0E0B0E0E80EF91E0A1F1B1FE092FA
:10743000AE01F092AF010093B0011093B101DC24D2
:1074400018C0D801C701B695A7959795879559D5C6
:10745000CEDE82E090E0A0E0B0E0E80EF91E0A1F68
:107460001B1FE092AE01F092AF010093B0011093A8
:10747000B1012197209709F0BECF7DC08090AE0169
:107480009090AF01A090B001B090B10196E4691660
:1074900009F05DC083E0F40180935700E89507B6DA
:1074A00000FCFDCF54C0F6E46F1661F5772031F192
:1074B000E090AE01F090AF010091B0011091B101E8
:1074C0007EDED82ECC24852D90E08C299D29F701D5
:1074D0000C0140925700E895112482E090E0A0E072
:1074E000B0E0E80EF91E0A1F1B1FE092AE01F092F9
:1074F000AF010093B0011093B10102C060DE582EBD
:10750000742423C0E090AE01F090AF010091B0016F
:107510001091B10116950795F794E79450DE682F06
:10752000C701F7D48091AE019091AF01A091B00155
:10753000B091B1010296A11DB11D8093AE0190934F
:10754000AF01A093B001B093B101219704C05524BD
:10755000772444244394209709F0A5CF96E4691634
:1075600041F485E0F40180935700E89507B600FCEC
:10757000FDCF8DE03CDE82E080936F009CC08334C1
:1075800071F40091AE011091AF0119DE90E021E09D
:10759000F8010C0120935700E89511247CCE833626
:1075A00019F5E090AE01F090AF010091B00110919B
:1075B000B10105DEF701E16090E021E00C012093CC
:1075C0005700E895112482E090E0A0E0B0E0E80EDA
:1075D000F91E0A1F1B1FE092AE01F092AF0100934B
:1075E000B0011093B10157CE8D3661F4E091AE0138
:1075F000F091AF0185E080935700E89507B600FC55
:10760000FDCF49CE823551F4E091AE01F091AF014A
:1076100005911491812FEBDD802F4CC0843421F52E
:10762000E090AE01F090AF010091B0011091B10176
:1076300016950795F794E794C2DD682FC70169D4C2
:107640008091AE019091AF01A091B001B091B101D4
:107650000296A11DB11D8093AE019093AF01A0933E
:10766000B001B093B10117CE843609F5E090AE01B8
:10767000F090AF010091B0011091B101D801C701A4
:10768000B695A795979587953CD4B1DD82E090E0BB
:10769000A0E0B0E0E80EF91E0A1F1B1FE092AE0149
:1076A000F092AF010093B0011093B10104C08B318F
:1076B00011F08FE39CDD83E08093E9009091E80076
:1076C0008091E8008E778093E80095FF04C010C099
:1076D0008EB38823C9F08091E80080FFF9CF8091B4
:1076E000E8008E778093E80003C08EB3882361F0B2
:1076F0008091E80080FFF9CF84E08093E9008091D9
:10770000E8008B778093E800DF91CF911F910F9174
:10771000FF90EF90DF90CF90BF90AF909F908F90B1
:107720007F906F905F904F9008959091B601892F50
:107730008F77813249F58091B7018032A1F0813293
:1077400019F5913A09F58091E800877F8093E80068
:107750008DE091E067E070E00BD28091E8008B77DC
:107760008093E8000895913279F48091E800877F52
:107770008093E8008DE091E067E070E05DD2809159
:10778000E8008E778093E800089582E061EC42E0A3
:10779000B5D083E061E842E1B1D084E060E842E145
:1077A000ADC084B7877F84BF88E10FB6F89480931B
:1077B0006000109260000FBE20E880E090E00FB6FD
:1077C000F89420936100809361000FBE81E085BF33
:1077D00092E095BF3F9A209A559AE1E6F0E0208327
:1077E000108247985D9A289A109289008AEF8093B8
:1077F000880090936F0083E080938100F0C04091F7
:10780000000850910108109201081092000894B7E6
:1078100014BE88E10FB6F894809360001092600067
:107820000FBE292F30E0F901E270F07091FD18C011
:1078300090FF05C0859194918F5F9F4F81F423FF46
:107840000FC08091090190910A014817590741F032
:10785000E0E0F0E0859194918F5F9F4F09F042DC6A
:10786000A0DF78941092AD011092AC010CC0DEDC68
:1078700036D38091AC019091AD0181549F4110F0BD
:107880001092140141DC80911401882381F78091CA
:10789000E00081608093E00025DC80E090E00895C6
:1078A000FA01923049F0933061F09130F9F485E1BA
:1078B00091E022E130E01EC087E291E02EE330E06B
:1078C00019C0882329F485E691E024E030E012C055
:1078D000813029F489E691E022E230E00BC0823069
:1078E00029F48DE891E028E130E004C080E090E0E8
:1078F00020E030E091838083C90108958093E900FE
:107900008091EB0081608093EB001092ED0060931A
:10791000EC004093ED008091EE00881F8827881FBF
:1079200008958091B60188238CF403C08EB3882318
:10793000B1F08091E80082FFF9CF8091E8008B7769
:107940008093E80008958EB3882349F08091E80081
:1079500080FFF9CF8091E8008E778093E80008954A
:10796000EF92FF920F931F9345D04CD008ED10E09B
:10797000F80180818F778083808180688083808117
:107980008F7D808319BC1EBA1092B40180EEE82E60
:10799000F12CF70180818B7F8083F80180818160E9
:1079A000808380E060E042E0A9DFE1EEF0E08081EA
:1079B0008E7F8083E2EEF0E0808181608083808131
:1079C00088608083F70180818E7F8083F8018081C9
:1079D000806180831F910F91FF90EF900895E7EDF4
:1079E000F0E08081816080838AE482BF81E08093BF
:1079F000B501B6CFE8EDF0E080818E7F80831092F4
:107A0000E20008951092DA001092E10008951F92AA
:107A10000F920FB60F9211242F933F934F935F93C2
:107A20006F937F938F939F93AF93BF93EF93FF9346
:107A30008091DA0080FF1BC08091D80080FF17C0C2
:107A40008091DA008E7F8093DA008091D90080FFE8
:107A50000BC080E189BD82E189BD09B400FEFDCF84
:107A600081E08EBB3BD203C019BC1EBA37D28091D5
:107A7000E10080FF17C08091E20080FF13C0809179
:107A8000E2008E7F8093E2008091E200806180932B
:107A9000E2008091D80080628093D80019BC85E014
:107AA0008EBB1CD28091E10084FF2CC08091E2004B
:107AB00084FF28C080E189BD82E189BD09B400FE50
:107AC000FDCF8091D8008F7D8093D8008091E10018
:107AD0008F7E8093E1008091E2008F7E8093E200B0
:107AE0008091E20081608093E2008091B40188235C
:107AF00031F48091E30087FD02C081E001C084E0A1
:107B00008EBBECD18091E10083FF21C08091E20027
:107B100083FF1DC08091E100877F8093E10082E0B8
:107B20008EBB1092B4018091E1008E7F8093E100C2
:107B30008091E2008E7F8093E2008091E20080617C
:107B40008093E20080E060E042E0D8DEC7D1FF91A0
:107B5000EF91BF91AF919F918F917F916F915F91C5
:107B60004F913F912F910F900FBE0F901F9018953E
:107B70009C014091BC015091BD014617570718F474
:107B8000F90190E044C06115710511F0AB01F8CF27
:107B90008091E8008E778093E80040E050E0F0CFDD
:107BA0008EB3882309F444C0853009F443C0809122
:107BB000E80083FF02C081E008958091E80082FD23
:107BC00031C08091E80080FF22C08091F300909145
:107BD000F200782F60E0292F30E0262B372B07C0EA
:107BE00081918093F100415050402F5F3F4F4115EC
:107BF000510519F02830310598F390E0283031050F
:107C000009F491E08091E8008E778093E8004115B7
:107C1000510531F6992321F605C08EB3882341F032
:107C2000853041F08091E80082FFF7CF80E0089531
:107C300082E0089583E008959C016115710529F49F
:107C40008091E8008B778093E800F90126C08EB31D
:107C5000882391F1853091F18091E80083FF02C083
:107C600081E008958091E80082FFF1CF06C0809105
:107C7000F10081936150704059F02091F3008091A0
:107C8000F200322F20E090E0822B932B892B79F7A2
:107C90008091E8008B778093E80061157105B9F653
:107CA00005C08EB3882341F0853041F08091E80013
:107CB00080FFF7CF80E0089582E0089583E0089583
:107CC0000F931F93DF93CF9300D0CDB7DEB7E6EBD2
:107CD000F1E08091F100819381E0EE3BF807C9F774
:107CE00024DD8091E80083FFE4C08091B60190918B
:107CF000B701953009F46DC0963040F4913081F1B0
:107D0000913070F0933009F0D4C02AC0983009F453
:107D1000A3C0993009F4B2C0963009F0CAC07CC043
:107D2000803809F4C6C0823809F0C3C08091BA0116
:107D300087708093E9008091EB001092E900209118
:107D4000E800277F2093E80090E025E0969587954E
:107D50002A95E1F781708093F1001092F10087C0BD
:107D6000882319F0823009F0A4C08F71823009F0A5
:107D7000A0C08091B801882331F52091BA01277005
:107D800009F497C02093E9008091EB0080FF1BC0AD
:107D9000933021F48091EB00806213C08091EB005E
:107DA00080618093EB0081E090E002C0880F991F12
:107DB0002A95E2F78093EA001092EA008091EB00A6
:107DC00088608093EB001092E9008091E800877F43
:107DD00051C0882309F06DC01091B8011F770FB70B
:107DE000F8948091E800877F8093E8009ADD809185
:107DF000E80080FFFCCF8091E3008078812B8093A6
:107E0000E30080688093E300112311F482E001C055
:107E100083E08EBB0FBF4DC08058823008F049C050
:107E20008091B8019091B9016091BA01AE014F5FA4
:107E30005F4F36DDBC01009709F43BC08091E8003C
:107E4000877F8093E80089819A8192DE8091E800A3
:107E50008B778093E8002DC0803859F58091E80039
:107E6000877F8093E8008091B4018093F100809136
:107E7000E8008E778093E80054DD1BC08823C9F4A6
:107E80009091B8019230A8F48091E800877F8093A8
:107E9000E8009093B40145DD8091B401882331F46A
:107EA0008091E30087FD02C081E001C084E08EBBC9
:107EB0006CDC8091E80083FF0AC08091EB00806257
:107EC0008093EB008091E800877F8093E8000F901B
:107ED0000F90CF91DF911F910F91089508951F93F7
:107EE0008EB3882361F01091E9001092E90080912F
:107EF000E80083FF01C0E4DE17701093E9001F91D2
:107F00000895F999FECF92BD81BDF89A992780B561
:107F10000895262FF999FECF1FBA92BD81BD20BDCD
:107F20000FB6F894FA9AF99A0FBE01960895F8944C
:107F3000FFCF4341544552494E4100777700080036
:107F400000000000000801120110010200000841B9
:107F500023360001000201000109023E0002010077
:107F60008032090400000102020100052400100112
:107F7000042402040524060001070582030800FF0B
:107F800009040100020A00000007050402100001B4
:107F90000705830210000104030904220341007253
:107FA000006400750069006E006F0020004C0065E1
:107FB000006F006E006100720064006F0000001826
:107FC00003410072006400750069006E006F0020BC
:0A7FD000004C004C004300000000CC
:00000001FF
